:020000040000FA
:02000000AC282A
:08000800A100030EA000831605
:1000100003138C1E0F28831203138C1A1028A72891
:10002000831203131A08A200303022020319482851
:100030003130220203195028323022020319582885
:100040003330220203196028343022020319682851
:10005000353022020319702836302202031978281D
:1000600037302202031980283830220203198828E9
:1000700039302202031990282030220203199828CF
:100080008514051586150616861606178613A028EC
:100090008514051186110612861206138613A028F0
:1000A0008514051586150616861206138617A028D0
:1000B0008510051586110612861606138613A028CC
:1000C0008510051586150612861206138613A028BC
:1000D0008510051186150616861206138617A028A8
:1000E0008510051186150612861206178613A0289C
:1000F0008510051186110612861206178617A0288C
:100100008514051586150616861206138613A02873
:100110008510051186110612861206138613A02873
:100120008510051186150616861206138613A0285B
:100130008514051586150616861606178617A02837
:1001400083120313981CA72818121816A728200E2C
:100150008300A10E210E090083120313850186017D
:1001600007309F0083160313F9308500073086009F
:1001700019309900043098008312031390309800CE
:100180008510051586150616861606178617A20110
:10019000831603138C160B178B1783120313D028A7
:0201A000D02865
:02400E00223F4F
:00000001FF
